:020000040800F2
:10000000C80600207D040008A1040008A30400081D
:10001000A5040008A7040008A904000800000000C7
:10002000000000000000000000000000AB04000819
:10003000AD04000800000000AF040008C90A000871
:10004000B3040008B3040008B3040008B3040008B4
:10005000B3040008B3040008B3040008B3040008A4
:10006000B3040008B3040008B3040008B304000894
:10007000B3040008B3040008B3040008B304000884
:10008000B3040008B3040008B3040008B304000874
:10009000B3040008B3040008B3040008B304000864
:1000A000B3040008190C0008B30400080D0B000885
:1000B000310C0008410D00086D0E0008B304000863
:1000C000B3040008B3040008B3040008B304000834
:1000D000B3040008B3040008B3040008B304000824
:1000E000B3040008B3040008B3040008DFF810D01C
:1000F00000F0EAF900480047FD100008AFF3008067
:10010000C80600200120D14908700020D04908709D
:10011000D04908704FF48070CF4948614000486171
:1001200080204861CD48008840F00100CB4908801C
:1001300000BFC64800780128FBD07047C54800784A
:1001400000284AD14FF48070C34948610120C14959
:100150000870BF480078401CBD4908700846007808
:10016000512806D14FF40070BB49486180200861D6
:100170004BE0B7490978481EC11700EB5171C9100F
:10018000A0EBC101B64A1170B1490978481EC117E8
:1001900000EB5171C1F3C701B24A1170B248114668
:1001A0000978405CB1490870AD4801788020084169
:1001B000AF490870AD48007809780840AD4908702B
:1001C0000846007820B14FF40070A34908611CE094
:1001D0004FF40070A049486117E09D48007851280D
:1001E0000CD19E48008820F001009C490880002026
:1001F0009649087080209849486106E04FF4807065
:100200009549086100209349087070470146052907
:100210001ED006DC052927D2DFE801F010121416E3
:10022000180008291AD004DC062913D007291BD18D
:1002300012E0092914D0FF2916D113E03F2015E060
:10024000062013E05B2011E04F200FE066200DE058
:100250006D200BE07D2009E0072007E07F2005E00E
:100260006F2003E0002000BF002000BF00BF7047E8
:1002700070B52025002405E00020FFF7C7FF7A496C
:100280000855641C0A2CF7DB774845704FF4B471AD
:10029000724800F081FE7148008820F001006F492B
:1002A000088000206D4924310880AFF26F120821C8
:1002B0006A4800F01BF900236F220621664800F00F
:1002C00045FA00236F220521634800F03FFA00231E
:1002D0006F220421604800F039FA00236F220321C5
:1002E0005D4800F033FA00236F2202215A4800F0E3
:1002F0002DFA00236F220121574800F027FA00232E
:100300006F221946544800F021FA00236F22092178
:10031000514800F01BFA00236F2208214E4800F0DC
:1003200015FA00236F2207214B4800F00FFA002333
:100330006F220521504800F009FA00236F220421A2
:100340004D4800F003FA002040490870FFF7DAFE3C
:1003500070BD2DE9F04305460C4601203B4908706D
:100360000A2094FBF0F000F0FF080A2094FBF0F163
:1003700000FB114000F0FF09C5F105004006060E24
:100380004046FFF743FF0746374887554846FFF783
:100390003DFF07463449701C0F54BDE8F083014609
:1003A000C1F105025000304A125C42F080022E4B2F
:1003B0001A5470470146C1F1050250002A4A125CE6
:1003C00022F08002284B1A547047274949780122AD
:1003D00082401143244A51707047234949780122D1
:1003E00082409143204A51707047012806D002286C
:1003F0000BD0032811D004281ED116E020211E4A5C
:1004000014321160102111601DE020211A4A1432AB
:1004100011601021121F116015E02021164A1032C0
:1004200011601021121D11600DE02021124A1032BE
:1004300011601021116006E020210F4A1432116072
:100440001021116000BF00BF70470000260000208F
:10045000240000202500002000100140002C014055
:100460002700002028000020B802002029000020DA
:100470002B0000202A000020000801400D48804782
:10048000DFF83400016841F4E0210160BFF34F8FD1
:10049000DFF82800DFF8281001600A48004770479D
:1004A000FEE7FEE7FEE7FEE7FEE7FEE7FEE7FEE724
:1004B000FEE7FEE79F04000824ED00E00CED00E0FD
:1004C0000003FA05ED000008064C074D06E0E06861
:1004D00040F0010394E8070098471034AC42F6D38B
:1004E000FFF708FEF4120008141300082DE9F0418C
:1004F000DFF8C4C0314B604503D19C6944F400640B
:100500009C614FF08046B04203D1DC6944F00104A5
:10051000DC612B4DA84203D1DC6944F00204DC61AC
:10052000284FB84203D1DC6944F00404DC618389BC
:1005300043F0010383810F2900D90F21224C4FF092
:10054000E02360450CD12261DFF880804FEA011C76
:1005500088F800C0D3F800C14CF0007CC3F800C19B
:10056000B0420DD16261DFF864C00E010CF1030CE2
:100570008CF80060D3F8006146F08056C3F8006143
:10058000A8420AD1A261114E0D01361D3570D3F873
:10059000005145F00055C3F80051B8420AD1E2615C
:1005A00008010A49491D0870D3F8000140F0804055
:1005B000C3F80001BDE8F081002C014000100240AA
:1005C00000040040000800402C00002019E400E076
:1005D00070B5194C8320206000256560A560174820
:1005E0006060012000F048F86168084360601449C9
:1005F0000D60086840F002000860206840F4803018
:10060000206020688003FCD5206840F08070206066
:1006100020688001FCD5606820F00300606060689D
:1006200040F002006060606840F48000606008682C
:1006300040F01000086070BD0010024000841D00F2
:100640000020024000487047001BB7000048704778
:1006500000A24A040549064A884202D00549884258
:1006600001D110467047104670470000002C014031
:1006700000A24A0400340140012804D0B0F5807F74
:1006800003DD012102E000202CE00021802801DDB3
:10069000012200E000220A44402801DD012100E09F
:1006A00000210A44102801DD012100E000210A4454
:1006B000082801DD012100E000210A44042801DDB1
:1006C000012100E000210A44022801DD012100E0AF
:1006D00000211144012801DD012000E00020084430
:1006E000C01D0001702800D1002070470121814009
:1006F0000148016070470000140801400121814059
:10070000014801607047000010080140012181404C
:100710000148016070470000140C01400121814034
:100720000148016070470000100C01400121814028
:1007300001484161704700000010014001218140E3
:10074000014801617047000000100140F0B53B4EC8
:100750003B4CB04203D1A66946F00406A661394E6F
:10076000B04203D1A66946F00806A661364EB042F3
:1007700003D1A66946F01006A661344EB04203D1FB
:10078000A66946F02006A661314EB04203D1A669A3
:1007900046F04006A66100240F2900DD0124692AE5
:1007A00001D0492A02D1032B00D10124032B00DD03
:1007B0000124692A06D0492A04D06F2A02D04F2A80
:1007C00000D00124692A01D0492A00D100256F2ACE
:1007D00001D04F2A00D1012503260222082915DA6B
:1007E000076802EB810206FA02FC27EA0C070760A1
:1007F000076893401F430760026889008E40B24338
:10080000026002688D402A43026015E0083947689B
:1008100002EB810206FA02FC27EA0C0747604768F0
:1008200093401F434760426889008E40B243426054
:1008300042688D402A4342602046F0BD00080140D6
:1008400000100240000C0140001001400014014063
:10085000001801400F4A536943F001035361936943
:1008600043F4007393610C4A136843F4807313607C
:10087000094B0A4A44331361516100219160916828
:1008800000F001004FF4565343EA401001439160D9
:1008900070470000001002400824014000000240A0
:1008A00038B5836843F480138360836823F460233E
:1008B0008360836801F0070443EA44438360124C79
:1008C000002914D0012914D0022914D0032914D0EE
:1008D0000E4C052915D0FF21FF2907D0204600F036
:1008E00081F80090BDF800004008208738BD012144
:1008F000F2E70221F0E70321EEE74FF08044022106
:10090000EAE70421E8E70000002C0140000800406D
:100910002DE9F04105460E462F4930488D4203D15E
:10092000816941F4007181612D498D4203D1816952
:1009300041F4806181610024FFF784FE0746FFF7E0
:1009400085FEB0FBF7F27000B0FBF2F0032801D88F
:10095000032120E00F2802D801240F211BE01B28CF
:1009600002D802241B2116E0392802D80324392199
:1009700011E0532802D8042453210CE06F2802D838
:1009800005246F2107E08F2802D806248F2102E07A
:10099000072440F2DF1144EAC40040EA841040EA30
:1009A000442040EA043040EAC43040EA844040EA4F
:1009B0004450E86040EA046040EAC4602861E86AA4
:1009C00020F47000E862193151434808A96841F0E9
:1009D0000101A960BDE8F08100240140001002403F
:1009E000002801402DE9F0410D46044611462046FD
:1009F00000F0D2FA032707230626681E4FF0040CE6
:100A0000012D01D0022D12D1218BC20007FA02F272
:100A100091432183228B0CEBC00103FA01F822EAF7
:100A200008022283228B06FA01F10A432283032D56
:100A300001D0042D0FD1A18BED1EEA009740B943E0
:100A4000A183A28B0CEBC5018B409A43A283A28B9E
:100A50008E403243A283228C012101EB800301FAF4
:100A600003F39A432284228C800081400A4322842B
:100A70000648844205D1B4F8440040F40040A4F88C
:100A80004400A08D401C80B2BDE8F081002C0140E4
:100A900001490880704700003C040040426B22F08E
:100AA0001F024263426B0A434263704705498A68EA
:100AB00022F001028A60C860886840F00100886006
:100AC0007047000000000240014800680047000035
:100AD000CC0000204FF0E0210A6942F004020A61D4
:100AE0006FF07F42904204D30A6922F004020A6147
:100AF000C008486170470000024A116002490001C5
:100B000008707047CC00002023ED00E070B53B4931
:100B100008883B4C82073B4DA4F12006A4F18000DD
:100B200018D50A8822F002020A800178012901D131
:100B3000006A804728888107334802D400882080D3
:100B400003E000882188401A3080288880F0020065
:100B5000288070BD0A88520718D50A8822F004023E
:100B60000A804178012901D1406A8047288881069E
:100B7000264802D40088608003E000886188401A1B
:100B80007080288880F02000288070BD0A881207B5
:100B900018D50A8822F008020A808178032901D139
:100BA000806A804728888105194802D40088A0807F
:100BB00003E00088A188401AB080288880F4007083
:100BC000288070BD0A88D206FBD50A8822F0100260
:100BD0000A80C178012901D1C06A80472888810430
:100BE0000C4802D40088E08003E00088E188401AC5
:100BF000F080288880F40050288070BD102C0140BF
:100C0000AC000020202C0140342C0140382C014045
:100C10003C2C0140402C01400348018821F0010197
:100C20000180024800690047102C01402C00002080
:100C300070B54FF08045288AC10740480AD0A9897D
:100C4000C90707D0298A21F0010129824069BDE83E
:100C500070400047298A394C8A07384904F18804D2
:100C6000A4F12006497916D52A8A22F002022A82A6
:100C7000012901D1006B8047288C800702D4A88EFF
:100C8000208003E0A88E2188401A3080288C80F0D4
:100C90000200288470BD2A8A520716D52A8A22F0BB
:100CA00004022A82012901D1406B8047288C8006EA
:100CB00002D4288F608003E0288F6188401A7080FA
:100CC000288C80F02000288470BD298A090717D558
:100CD000298A21F0080129828179012901D1806BBB
:100CE0008047288C800502D4A88FA08003E0A88FBD
:100CF000A188401AB080288C80F40070288470BDD0
:100D0000298AC906FBD5298A21F010012982C179D7
:100D1000012901D1C06B8047288C800403D4B5F829
:100D20004000E08004E0B5F84000E188401AF0801F
:100D3000288C80F40050288470BD00002C00002016
:100D400070B543490888C20742480BD00A1F128871
:100D5000D20707D00A8822F001020A808069BDE824
:100D6000704000470A883B4C3B4D04F190049207C9
:100D7000A4F1200618D50A8822F002020A80017A1E
:100D8000012901D1006C804728888107334802D4AB
:100D90000088208003E000882188401A308028885D
:100DA00080F00200288070BD0A88520718D50A8892
:100DB00022F004020A80417A012901D1406C804767
:100DC00028888106264802D40088608003E00088D5
:100DD0006188401A7080288880F02000288070BDCB
:100DE0000A88120718D50A8822F008020A80817A38
:100DF000012901D1806C804728888105194802D4D7
:100E00000088A08003E00088A188401AB08028886C
:100E100080F40070288070BD0A88D206FBD50A884D
:100E200022F010020A80C17A012901D1C06C8047EA
:100E3000288881040C4802D40088E08003E0008800
:100E4000E188401AF080288880F40050288070BD26
:100E5000100400402C000020200400403404004016
:100E6000380400403C0400404004004070B5434951
:100E70000888C20742480BD00A1F1288D20707D041
:100E80000A8822F001020A80C069BDE8704000476C
:100E90000A883B4C3B4D04F198049207A4F12006CC
:100EA00018D50A8822F002020A80017B012901D1AB
:100EB000006D804728888107334802D4008820804D
:100EC00003E000882188401A3080288880F00200E2
:100ED000288070BD0A88520718D50A8822F00402BB
:100EE0000A80417B012901D1406D80472888810615
:100EF000264802D40088608003E000886188401A98
:100F00007080288880F02000288070BD0A88120731
:100F100018D50A8822F008020A80817B012901D1B4
:100F2000806D804728888105194802D40088A080F8
:100F300003E00088A188401AB080288880F40070FF
:100F4000288070BD0A88D206FBD50A8822F01002DC
:100F50000A80C17B012901D1C06D804728888104A6
:100F60000C4802D40088E08003E00088E188401A41
:100F7000F080288880F40050288070BD1008004060
:100F80002C000020200800403408004038080040B1
:100F90003C0800404008004070B504460D46194921
:100FA00019488C4203D1816941F400618161B4F137
:100FB000804F03D1C16941F00101C16113498C42E5
:100FC00003D1C16941F00201C16111498C4203D1D1
:100FD000C16941F00401C161FFF738FB06462046B4
:100FE000FFF738FBB6FBF0F0B5FBF0F0010C4A1C44
:100FF000B0FBF2F02185401EA085A0841120208046
:1010000070BD0000002C01400010024000040040B0
:1010100000080040044801688907FCD5416841F098
:1010200002014160704700000000024002E008C871
:10103000121F08C1002AFAD170477047002001E052
:1010400001C1121F002AFBD17047000010B54020DB
:10105000FFF72CFDFFF7DEFF2448806820F0010039
:101060002249886000243BE0214800EB041080689E
:1010700060BB1F4800EB041001681E4800F0DCF85C
:101080001B4901EB0411C860194800EB0410C0684B
:101090001949884223DB164800EB04104068401CC5
:1010A000134901EB041148606420114901EB04115C
:1010B000886000F011F90E4A02EB04121179621CEB
:1010C000D0B2FFF746F900F08DF808E0084800EBD1
:1010D00004108068401E064901EB04118860641CFE
:1010E000042CC1DBFFF70EF810BD00000000024029
:1010F000D800002038020020D3450B00FFF7B8F8D5
:10110000002014E000212D4A02EB001251602B4A0E
:1011100002EB00129160294A02EB0012D1602849CB
:1011200051F82010254A02EB00121160401C0628DD
:10113000E8DBFFF74DFA2348FFF7CCFC22490920F2
:10114000FFF7DAFC48212148FFF7E2FB02211F48A4
:10115000FFF7A4FCE12203211C48FFF7A1FB1C4977
:101160000020FFF777FB02236F2200211948FFF7C9
:10117000EDFA41F698111848FFF70EFF174A0221C1
:101180001548FFF7B3F94FF4347203211448FFF701
:1011900029FC4FF0E020006940F001004FF0E02111
:1011A00008610846006940F0020008610120FFF76D
:1011B0001CF90020FFF709F900BFFEE7D800002066
:1011C00000000020407E05004D1000080024014072
:1011D00038020020000C0140000800409512000871
:1011E0000004004010B512490878FFF7F6F81048DF
:1011F0000068401C0E4908600E480068401C0D49FC
:10120000086008460068042801DD012008600848DD
:101210000068032802DD00200549086004490878B9
:10122000FFF7D3F803490878FFF7DFF810BD000097
:10123000180000201C0000202DE9F04F4FF0400264
:101240004FF000034FF000044FF000050F4FDFF8A0
:101250004080934212D030F9139003FB01F606F060
:101260003F0637F916A009FB0AFB5C4438F916A0C3
:1012700009FB0AFB5D4403F10103EAE784FB041068
:10128000C5FB0510BDE8F00F00BD00002C3E0008B6
:10129000AC3E000800B520B41248134A1168134D43
:1012A0002D684FEA4505A94214DC435E01F10201B5
:1012B000116003F5004310B440F2CF2403FB04F3A4
:1012C0004FEA234310BC0A4803600FB41846FFF7E7
:1012D000DFFB0FBC20BC00BD00B5034A4FF000018E
:1012E000116000BD1C130008D40000201413000876
:1012F000D00000202C3F000800000020D800000093
:101300002C10000804400008D8000020F005000060
:101310003C100008881500005B00000001E5BA5091
:10132000C6FAF32A40A4D8B563747EAA6430B03FED
:101330000080F233D15892B0EC1197146594AA4B07
:1013400068EF38E32C6064AC6A3861132BE42A53ED
:10135000B0A933E6791A24C8452051F7C6E53F3EC7
:10136000F9CCC0F1774CFBC3FE1ED95953D861EAC2
:101370004DE46E0F3D1ED4DE96067FE5F9E5AC1513
:1013800068C2BEF795496FCCA50DBD546FF40F2010
:1013900084CD60D79B3FDFA920081154F9CFE5F237
:1013A000B60E38F9F300FAF34C15C336E5DE8201C8
:1013B0006AD0CCCA0D517FF8EC10972BA9BC81DB09
:1013C0001E26D2D2DAFE342041CBAE493F137AA793
:1013D000B5FA72E8C2F8F5376BF57FF9B71D93E8F7
:1013E0006F378FFEC0C7A24A67DDBFF42615BECF98
:1013F000B53FE4FAABDA3C25230C59FAA1E3FFC26E
:10140000E92115ED6FCBCF7AD4CA14EE4D0D4DA264
:10141000FF7FDFFE19D87B7809BF24DF56F36BF31B
:10142000CC346DBF3FD6FA3336C493D53A2C62CE56
:101430008640701BE4CE5166689C6500C446B3AF1D
:10144000F44FEDC84DD0B3485306841F75D56FE3F4
:101450008B27C6FDC2109E1D01D065FCD61348E542
:101460007D4441E167C924087CDCDE2DC5ED93FE97
:10147000B0157CDE8E044718F011FCE9D5F140BAB6
:101480006F1FB3317CA1FF18CD404CD22AE8465BD8
:1014900061D29CD0CD5767B6F609402759E54E1D5D
:1014A00072FB1224D8C9D1DB902200EABC03130BD3
:1014B000CF0D27FB44137DF145F74318FBDAA3EE6C
:1014C0005DD08726013D0BC91D15A025430141CCE8
:1014D00072FD623AFDCDD905060A3E068B25CCC7C2
:1014E000A9FAA939F9FA79982848E5490B9C223FCD
:1014F00056B5C9ECE84EB6B83F2C88F86F0DC5ADAF
:10150000181AFF7F4BAEAE36F5CE3602D904B3DBE8
:10151000E35476BC492356E0D7FB0A21FBB056348E
:1015200078F342F2501548FB69D4192C9F1896AFF6
:10153000F87B6ABC4BD9366CC5C3070908EFB1FB11
:1015400076D0542CF50C1EBB454D5FF120F012F9FE
:10155000820098E6F10C9D0A51E27B3870F0F1F8B8
:1015600063061BF6BF09F0E42D085F07C7F49A2F46
:10157000C7CB800B023575C098FC0EFA85F271EE70
:10158000583F9109E203612887BD6401C5FE77F7E2
:10159000C1ECD80AD7F982EC462FABDCCF0F38105C
:1015A00062A3A411C224D7CFAE0D1D2B78DD34F772
:1015B0009C3B03B3F90C473F47AE9D0EC72338F65B
:1015C00057F1822967F4E3E91A1361D3AC2B871131
:1015D00055D11E13940D8BE611285C1678C81E2871
:1015E00028F7ABC53948DE031FCC2A13501402F587
:1015F0007BF90016FEF657F131DE2808630A17F66C
:101600006830DAEAD50362F62DF24208F5F6AA212F
:1016100098BCC2F9D51C5C005F06BEE5B02DB6CD06
:1016200082E9642FCCF0E108C4193FFD8CE0BE3B99
:1016300043D4A1E0A2480BC7B7091AFB54132A2CC4
:101640007FE37D0688F89314DDDB380EE51E10C6B7
:1016500005124609A2DF9C11741ED9C57612F31536
:1016600065C0403ABFF48BFFE3114EC7B53A11E8AD
:10167000BE0E9E307BCDD30F59E4E6048C0F5FF392
:10168000292DB403A6C9D615571D1BCA373CE7EA56
:1016900070C63A304BEBAE1E41F54DF848FE62E1A4
:1016A000302076E8AC15FA09B20A0E108EC17E140D
:1016B000A21CA3C5D200E727D1C2BC2FAE1F26D6DD
:1016C000A63596C56F0C901030E0E241AFD91DEF02
:1016D000F63347ED8AEC9426D1EED1EC0A0D6DFE7F
:1016E0002A14C4DA350AA50EC6E67C0A84F8C806B0
:1016F0000001911DB1FBC2B93824141814C5513A28
:10170000A10C78B5052985F299F55A1F59D3C41C47
:101710003EF01DEBBD3FD0E00DFF620B72D39CFB92
:10172000280917209109E5F1822D98E6F4D26A4F35
:101730007AE98DDF1320FADF3A1939092918380EB2
:101740008AC1F90D41F6BDEA972996F2A3EF16106A
:101750005BF3CF0D21EC3FFFFC2A82AAC101CF0E23
:101760007EC0E546E5079DDF19FFCCDF391C1E1161
:10177000D7FC921930E360EE8616E6EFE7FE0B0623
:101780008E0388F53CE49327660C58D7472A15EA60
:101790001DD7CA3E44FC4A0735064BEDA4FE49F569
:1017A000D73C1F0B34E4512569EC81EFD229A0E529
:1017B000B30587FEE6C47832B3092E00163BA1CEEE
:1017C00032D7A10CAEF69607D7258B10ECCE77F763
:1017D0009A3010EE26FDD30FD8C84E09181996F08E
:1017E000241D02F530F523F98AEDDF14EFEBD3F871
:1017F00069FEEAF16F209FEBDC0D982629AF850783
:10180000A025CBCE8531F0121BCABC190B082BE5E5
:10181000B4182808B2F9E602B2F6721047002EFF9B
:10182000730DCAFBA2F0F6F1451FC1FE8BEA021E42
:1018300096DCE7E70128AFF05CFF331481038BFEF1
:10184000CDED97008A0253F18726FE1D09E9261483
:10185000AFEE65EBF8FEB8ED880A44F98D1C3A1737
:1018600043E949F88E031EFE73F9FE0BCD0247EDE6
:10187000D006CF0EB6F80A0BC40439F1F8FC71EEAD
:1018800011FD390B52F5E82290F7DDDA512415ED00
:1018900047EE681850FF53F1300B37144FF0140423
:1018A000BEFBA2F371FF200692040800511080F4E1
:1018B000C3F32CF44314501407DEFB1672FB73E4DD
:1018C000B402950AB71CD0E05800340E65FC11151F
:1018D0003D09CBE16CEF9B1785DD730EB015C2F9A6
:1018E0004BEC91F33D2037E9D601B8186A0D4ADC7C
:1018F000DA02470259FAFB2E37E9FA06EBD49DF7D4
:10190000E51EC3DF2323DBFC9AF3020CC9FFB5FA03
:1019100051F8340E45F61915ECF9C0F08E1931F373
:101920009D0C61E88CF612109F03BC057BF7F50D4A
:101930004FDA56080D1244FC570649E33C0F3601B6
:10194000BB07D80A85F17004CAFD200802F6D3113E
:101950002E03AEE2BE1080F579053A048C0CC40863
:101960007BF8D2FCDCF67A136FE10F1CCC0759E848
:10197000021F72E5C502AB05A9F8E4FA61FFEA03AC
:101980000AF6EB12F608B708C3E036ECDB125EF697
:101990003E1925EF61FDEBFE8A04D227F6DB520CDF
:1019A0000AE335F01F200F0ACD182CE20C018FFF3F
:1019B00091F541F7DA187500EFEB4E20F2DD1E13BA
:1019C0008A041DEDF61BFBDA2E027AFF2D06BB1DE5
:1019D00094FC43EC7AEBEF17FEF5BE103E05F4FBEA
:1019E000860259E87D1768F03E1AD0F5A7EDD613A8
:1019F00050E96A260EF7FCFED2006FCA83119120CF
:101A0000670837FEF4FEF3EDBC044703E5F38519E0
:101A1000B9D53B163D0AB7F4602DDBCFBC032BFADA
:101A200076FF9B02A4FE24205CFF71019FEA4E0812
:101A3000C5ED96078009B6F5BF0C66E3DC22ED081C
:101A400062F74D0C36C4951E98F9F8FF842228E100
:101A5000662506CAE315B5FEAB18510D2CB6DE405F
:101A600098CEB4410AF8AEF3322E809F751643FE2D
:101A7000D020941133FE05E9F1DF7E13B0002F3B37
:101A8000F9F90AE14BEC0CF0BE0D5B1A0E2220F0C6
:101A9000A8FEABC73CFA741D200A543DF7D547EAAF
:101AA00095F4AE09F9257A14EBFE37D4A0FB03DBDD
:101AB0008E17BD16990BA90D64D861FF11EA5D124E
:101AC0007C1F5B08210116D1D8F4A1F9181C741EE3
:101AD000BBF4CB0C6ECF3F0216117406BF1D0AFA81
:101AE000D7F8FBD90511B9E66419DC3715D5FF0520
:101AF00049E178F5B415B81AEF146EE865FD24E0F5
:101B0000D40B5D134A0A6017CFE31D04DCE0F60531
:101B10000B1D0A0BFB16B7DBDDF147EBC113FB1AFC
:101B2000EC11B9FE33D23F0164EF8A150D272FFE69
:101B30000EF9D3E443EC09FCF61DE314570484F4D6
:101B400072CF43028310AE1F541550E9FEE0A9E2A4
:101B50000D148C0F652A64025AE1EBECB6E3FF1B0F
:101B60000A0D7C1EFDFA78DE2DF180F4BA23340DC7
:101B70003A1712E2EBD58E052600C432990D2FFDDF
:101B8000C7DF05E5C6126C04B527DBFD5EF726E965
:101B90006DEDAC158104C2243CF811EA19EDD1F0C9
:101BA000421BF90DFB1AEAEF25EDC4EEE0F8152A09
:101BB00054FEDC0CEDF3FCEBA5F896048F12A800A4
:101BC000AF1C77E10FF4EA04A2F2891BE00EDBFD03
:101BD0000DEB02F5D3FBAD10E714D7F80403B4EA1C
:101BE00001FAC007600092198DF371FF35F32CF5EF
:101BF000630A5C02BD148DF2BBF5BFF59D0D59FC67
:101C000071013311F0FB180711EB2D0423FBE00DDC
:101C1000B30883E4BA0E8CF6D8F3FA1B970285F268
:101C200061FFC6FA16FBB5107901DBFD5A0971EDAB
:101C3000F204A8FFD30EED09DEFFF8FEF3EA8009F7
:101C400069FE2E1775002CF8D4F6F3ECF50D680438
:101C500083104B0497EAD6EBFB01800CDF117F0E5B
:101C60004CEAB8EE9A0423FAF317790530F5A8FD8B
:101C7000C4F2E2009B0347172CF8890630F458E9B8
:101C8000CA10A4FE8311530413F4BBF33CFAD40925
:101C90007F0E4F01B6F595F3E4F8D907EF13D600A0
:101CA0007EFD11004EF4AB0340FC170D9E07B804F7
:101CB000FEF43DF467082AFE200A7E0190FAD0F572
:101CC000E3FD05FD6F0D6708B5FC48FC49F8B00160
:101CD00004FF31056C043E0306F9F0FC23F9740699
:101CE0009D0B15021AFEA5FB63F5FCFF340CD3FB1C
:101CF000BF088CFA61FC27FC8A049F003202350A77
:101D0000B7F20800E0F7DA00E00D3105FC0065FCF1
:101D100046F17EFE7409DD075707B9FC55F8BDFD95
:101D20001AFB9300381044FDBD01DBF902F84205AF
:101D3000380C07073BFF74F453ED2D07CC07620FF7
:101D400081045FF27CF55B0511FEB3081B0E9EF368
:101D5000970087FAA5F778093D0C7A00C90089F346
:101D60009EF1AB04120D730ADE0252F401FAC003B5
:101D7000D6FE280B09FC65FEA5FB69FF420569013B
:101D80008E047101D1021CF13CF9B0024A0A1E1006
:101D9000A4FE03F3A0FB66FAC904FD0C16FD06F9C8
:101DA000E3FB87FD1D033D08BD004A0622FEE8FA5D
:101DB00027FBC5FE8E02FE095705B6F6CBF977F66E
:101DC000060E280BA4FFDCF7DBFB9F01F303B00139
:101DD0000EF771FF10EE4BED7EFF100644108037BA
:101DE0009230351EC00664D75DE7A5E30BDFBCEE7D
:101DF00088F53E07800AFF1ABB1D18F3C8F30000E0
:101E000056F6E7FF541403F13CE68F1159F9D00759
:101E1000380D12F9DD082310BFF57AE89A0413F3A0
:101E2000E908AD0F1BF5EE032A01A2077103B9FC07
:101E3000BEF70CED6BF52504F207010E8E164DF87A
:101E40000400CAFB00FED8F512FCCBF564EF0A21B2
:101E50005EE4A13AB9FEDFD1A61E03DC8600D3FA08
:101E6000EA06B9FC4A1D421949F77AFD9DDF52077F
:101E7000C2254CD147EC1F0C93E78D4961FEA9F9AF
:101E80000B0725EFC2E4FAF1B5FD94F86C30F3EEE0
:101E900078201C09A7F062F774F188F751FA33FD36
:101EA0008AEE5635E80FB0FF4B02CBE1AAF32B12B6
:101EB000EEF2B8021C096BF744103A0206F853061A
:101EC000000079F0FA094CE8300BE314BF08410C2C
:101ED000D4F65DE573F64F170FF6B81626FEECF84C
:101EE0004D0F1002CCF43A046AFC23FAB70696EEC2
:101EF00085053A05A207F0FBC30903F2E200670774
:101F000037FC740966F7E700DFFB6804D8F6EE03D8
:101F10005EF9E711930045F87C07F3EE5E0C0304CD
:101F2000F5F67CF2200A0110FD0CC3F641F4AEF385
:101F300076FE3B0184F61A10390AB309630847EDAF
:101F40000CEEAE0CF9F79C0F4CFF9AEF2D08310701
:101F50006B0B6002CFFAEAED0BF3B9FBA90D740726
:101F6000900C1C059F0292F149F841F551FB701C41
:101F70000EF99B0376FCA801170B3A06E1F336EB4A
:101F800082FE7904D907EB13E1072CF8A80092EE42
:101F90004DF724F5000121022F0F890654FD670932
:101FA00058FFAF043AEC34F633FB69015D141C08AA
:101FB00066F9BE0E4AF2F0FC3604D3E4310780091C
:101FC000AA0851FB8F0040FCE00DDFFD78F16C04A6
:101FD00083FC3605D30E630615EB060A5FF3D2FCCD
:101FE0009D0B9EF293FD700843FEC101BC044AF2B2
:101FF0009C126FF6C0044810C1ECCAFD2F10D3F933
:10200000AEF8611227E4D2FEBC1A17F8C6FABC0675
:102010000B08B5FBB5E7F300F90F24F4020A5014DE
:1020200069EC4AF3C81B49F5F0F95706FBED32029B
:10203000380D371400FE81EF81F11914F3EDAFEF85
:10204000F9250DEB1005561EB7F4B4EEFC0015FE95
:10205000170ACCF3FDFBE313B0EB8B10071AF2F178
:1020600063E0E107A30481F0E108A4FFB31B7EFE57
:10207000E6EF1612BAE1A6077B0E53F165FD59FB98
:102080007119F1F86F0B92EF74F43BFDBD01391F2C
:10209000E2D9BE109607C102D80880F394FBEDF791
:1020A000660C4AF3100617F89B036419DEEE6BF713
:1020B00073F7DB12E50723FB660D9ADBD1045305AA
:1020C0001B0C8FFC77E2FB181004A50F7CF5F0F9D0
:1020D0002CF35207B51459E82BFBCDEFFF1AA20AD7
:1020E0000DFEBB083DDFEE0533131FF99EF22600FF
:1020F00074083D0B59107CDF4607E8F800FE062205
:10210000C7E1821546F1761490F7CAE79C138FEB6E
:10211000E61737D2A5370EFAB8ECAB317BCC0B1EE5
:102120008BD232014B1AF4FD5C00E5F3E83AF8E992
:1021300003086DC08D09C62490CFE04EB2CABC180A
:10214000CFFA8EED29193FC09C3EF5CB513AB0FF36
:1021500029DB4D2312D0A53A22D25F1CA6DE401106
:10216000C70B2DDCC63D78B4EC50DAEAA7EE3BFC99
:10217000C7DFB73451CDCC1D0ACD2918781FA5244F
:10218000174C669062F988CD9206613D130B53306F
:102190006EBA990DE5C92A13402498E339348CB9F5
:1021A00069282FFBDA012906E2EE02F4FEDFB24BCA
:1021B000C2BC9C2541F434F8594FDFA8332832D9EA
:1021C000B4EB1F367C0B1E12E7C0840B85F36A3C10
:1021D000AF06B2E05D14DFA8B42DECFBB819B6F978
:1021E0002EECC52BAFEE7323DAC03A189BEA5303EB
:1021F000B6247BB8882446080235060A6DD5E5DD8D
:10220000AACAD12EE40B87101D04D0F2DD30E7E816
:10221000BC0643EA4ADE9F03AB06E909A9F8553933
:10222000F302AD105ACABFDFC21027E54F2E2DEEC4
:10223000EF00F1F66B21C81BFBD9EFFF13DE87100F
:10224000E1F282019C2528F5222AA1F7F7EE45DF6D
:10225000B1E683244EF5201CD9EE4A088A1799F47A
:10226000DDEF5DE6F00EB8EB851AF8EA911CD506B5
:10227000FCE8BF4AC1BD7AEAFE0897E9792CDBF990
:102280008CF71D198DF527FCA910E9E07EE86A237B
:1022900084E065291B0DFAB2AB4591F5BC021F0F16
:1022A00021DAC9EEEFFF68035815662537BEE8232B
:1022B0004B00B3DBFE2113F74BEB241D12FA3ED982
:1022C000F93AF8E80AF7262A16D026FEAE1FD4DD22
:1022D000313096F1A2C7633143EB48FCF93813DE85
:1022E000DFE83326F3C24F1BEF16DCE05A1F5C0019
:1022F0009BEB060EDE029DE32F28C2D1A2F56735C7
:1023000084E1CB0EF538FBC254EC622224C72627A9
:10231000E311ADE5A21EE6EC46EFAA35B3DC90F979
:102320004E1C9AC416103A2E55E3D615B4190BB4A8
:102330008820D1EE9CFB3C23A9CFCD18340EA1F709
:102340009E098B27C4C61804631C0EB8472EB20B17
:1023500014F29534B1E4B1E7240BBAE5EA1A83101C
:10236000C6D08908882132D8082CA20A00BE8B2644
:1023700065FC1404440F3CE648FD7A1475EB0B0829
:10238000501554D3222A5401B1CFC92B76FC44E412
:10239000A429D6EC0FE02C205EF5A415170A60C224
:1023A000AA1FB309D0F16B344DE299DFA412ADFD41
:1023B000DCF43A1BE5F2A7EDCB21E2D9B3082D1AE4
:1023C000F5E1C625CEE9CAD39A3214EEA6082A2A28
:1023D0000ACBE3E6F7154E06A3040B1DBBDE9DF901
:1023E0002F1128DEB528D8F481F1152C85D901E606
:1023F0005924F0FA0707CC1BC3CA01FAD51C06F909
:10240000E11BEFEBBBE0C7200AF642069D20D2D2CB
:10241000F6F2A21D6CF2C1014C13D6D79717BC1966
:1024200034CC9312F2F15EF9A61D29EFAAF5461AF3
:10243000712C340B9EF397D69B02B7F11DEB8D34B4
:102440006AE675EFD00994FC4B1921052DF2C9FFFE
:10245000C70A05CF351C120F13DED049BBDE8AD860
:102460009F2C2BE4C2F8B926B8D97CF2A92643EBFD
:102470003D1FEA0367C976263E048DC7CC1FAB0417
:10248000F3EC5C2D8FE733FF6732E8CCB3F3E7164C
:102490006DD7CE13E00F35F4862C4EF48CB8633232
:1024A000CF100ACFC02D6FE0C5FF1C31C0DA9C0FE2
:1024B000941125D87408AC0174DC5E243B1412E539
:1024C000FE1F6DEB9ADDC52C22EAA0FDA719E6DB05
:1024D000E00D0B1B5BF33C0D8AEB45E23A1B07F466
:1024E00046083A1B81F198FB9E078AEE5DFAB5110A
:1024F00090F74302A0FFC4EE8D078D1EE1057CF529
:1025000012E577F8800817F49A1B58006AE5BC18A2
:1025100030F7AEF5BF1FC2E72BF95E0D3DF32FFC80
:102520000F0A76FDEA03520CB3DDF315520A49E4B3
:10253000251924F15CEBB01876FE47021805B2F6B7
:10254000DE026EFD12FA3F014E06F7EDAC17EFFE0C
:10255000C1EA531B8EEEEA02B110C0DC7EFF0926F1
:10256000ACEB7E00E80EA9E49713EB126FE1F410D8
:1025700073F546DDC12AB5FEB803AA0CE3E7640291
:102580007406D5ED25051F0DEAF0840A09FEF70152
:10259000A0132BF94AF3F4FD2BE407055524F8FBAF
:1025A000CD0037FFC6E59F034413A7EC7610F4FB7C
:1025B00032EC4B17F8FBA0FC410C03F32FFC6EFC34
:1025C000E6F0B81618072FFAC1FE1101B7F4D103CF
:1025D000D506A0FF29051AE4DC0B5B05E8F9B1126A
:1025E0009F0030F98E0405E97DEE9825420681F1C1
:1025F000F10ABFF6FDF7B111A9F8FCFF0EFAD0F110
:102600003D0AA90D50FDE3FEA0FD91F2170B99F4D0
:102610006806730D14F1D104E4F83DF6F3175DFE7E
:102620008DF2F41325EF24F1BF1EB9FC47EC3F13E4
:10263000C7E300FE41221DED5F08E202F2F0D00781
:10264000C404D9EE0707DD0751F8680527FC58FFD9
:10265000A50E76FDF6F4AF04EAF12C094F05BEF89D
:10266000910A34F99F02300CB4ED7CF3BE10D4F41F
:102670003506481470F14204FB0566E56709D40B82
:10268000ABF0BB0B21057CF42EFF93003D0C980EA4
:10269000ABEEE1F491F58FFDFF04730C030594FBA1
:1026A0001501F9FA7A12CBF55802AF04F6F34AF1A4
:1026B000D1EE6A11641AB111C6FB3B001EE6FEDFC3
:1026C000590F9C1180F32A0257059204340FDE0340
:1026D00012F9CAE83AF0F9F85C15F8119D0C4B05AF
:1026E00027FC4CFC7FE4D8F75C0346F1AF08AC153F
:1026F000CEFCFB1911FE09E60C0208EBA1F67116DF
:102700007A0026FF9F18A702E3FF61FBF4E7DDF1E3
:102710000304A8FDF10A3D0BC903031927FC81EF4F
:10272000C8F082EBEB01400FC5014B04240BEA0219
:10273000F60537FF76E9A1F76EFA23FBAF1DD8F552
:1027400066F9751978F52808FA0907DD840AD101B8
:1027500096DA181AAC1644FB4608E50990E40AF923
:102760000E0D70F158FF5EF67903B4041B0B741C58
:102770005DFA3FEBA0FDDDF091F408179604E3FC51
:102780001B0AD7F9BEF8D006B306E204E5F27AEAEE
:10279000CEFC3D098505E11CFF0403D9EA03530281
:1027A000EAED910ABA0C94FBB1123B120EF852F604
:1027B000AAF6F9FAD2E911E71113AC13CD020F20F2
:1027C000E3FE22E80EF90EF71EFD8FFED103AB03E8
:1027D000F8FDBC05BB1C22FC53F03BFFD3E4B2F573
:1027E00048104E0AA400660C5A0A56F565FF9CFE76
:1027F0002BFC1CF3C8F37C0BA6F5410C5A20C0043B
:102800004EF492EE20F3B1FB2A023700230C63F55D
:10281000FB01060BBB087B0D85F32CF59EF49B0199
:102820008FFF570761FC38F6B514A607B7F377F8A2
:10283000A2F20AFA900F97FEE6022D05D6FFF8FFE6
:10284000C80523F941F3AA0893FDE2038D07A6F218
:1028500015FFC30C74F2930076FF000187FCAFF202
:10286000D51AFBEF4AF3301FDCF4B900AA0C78F359
:1028700059F973F8A10DB9FFB5FBDC0D29048EEDF4
:1028800001FAEB1277F88CFA7BFB1EFCB2F7711899
:10289000C70CA6F3F30166FA4DF9DAFF0B0946F30C
:1028A000EA03F0FC880A3BFE0FF6A10E2FFDD3FAD7
:1028B000E9F4C7F502F8D2163F1433FD24F42A02D6
:1028C000F4FAC4065B0563F41FF817F8811B61FE78
:1028D00082FFC5FF9B016AFA4AF368047BF7420650
:1028E0008C0C2D06A6F31C0900FE6401BEFA72E9E9
:1028F00082016709F3171407790202F428F53EF103
:10290000CAFA33FD9B014C1197FE2F0F11FD02F700
:10291000E0F990F85AF8A4FCF61CAC141AFE5DFD20
:10292000B7F1E7E916F97EFF130CC6FA9108FB1917
:1029300098FBD4F64EF133FEECFBC3F63909410B9C
:10294000680335096C038CF9A4FD0EE302F7C61287
:102950005A0BE6016D010910A0FE0EF853F017F7AF
:10296000D7F950FE65111807D80A27FA05FCC100EF
:10297000D1EE08014302F8FEED0A1AFD18065E0BBF
:102980006EFA87FEEEF11BF78A00E7FF5207C007D9
:102990008FFC0802F205FDF9E3FC53EF670A3E06DF
:1029A000D5EF8FFF340B2C0DA1F94205C4F15BF27A
:1029B000DD07BB0B8DF454E9042ABB1E42D9B9D103
:1029C000292DDE2E92DBDFE5AEF7B511EF1363F2B2
:1029D00051F853063E06B3F103F1CC1DBB0A18F3C0
:1029E0006EFB5BF092062A15790265EA5DFDA30194
:1029F0001D02170AEDF3A90D520844FA14EECDEBAF
:102A0000841FE9092CF8EA0418F2C4EFE1096818F8
:102A100037FF3F02FFEDCEFE7FD102B8FF7FF850B7
:102A20000080FBB0FF7FFF7F008000806B61FF7F35
:102A3000340B00801C09006D1CF3C807A58FD2FC65
:102A4000FF7F99E106CA29DAC9155D527140CA9122
:102A50000080FF7F9534FD9048128FD3B93D7F25CC
:102A6000B6E2A2B2B621A25F0080F0282032E8B917
:102A70004D3680F616F906DFE932C3F68EB0FF7FD9
:102A800002CA3BC08A2E92D70C30ACFE000095CC17
:102A90004E1DE729E1B2E15D0DD426BFD54678F59C
:102AA00033FB77E3E91F0A0BF4FC1C057BB77A289C
:102AB0004E1DD8F3BF09BFE065FC1C09C03120F0F2
:102AC00069D305258DDF4300FA1CF1F5570472FD2B
:102AD000ED08F0D1AD25EA1A3FBE4C3F8CE4A4D5F9
:102AE000A32C06F76E0EADFC4D0FF8D271FF3B41E3
:102AF000F9BA59268D06FDCF8B2646F3510D6FF49A
:102B0000A90EEAF1CAE95F1D25DB252F1F0CF7D7B7
:102B1000D904020BFB017AEB851CB3DAE2003F28F3
:102B2000A9E35815F8FD91F62EFFE203ACE945F54F
:102B3000503F56DF03F0BC3010DA43ECCA1334F6D2
:102B40006F0C070796F08DF3DC1F1A13B5D0951D97
:102B5000FADEC7F4373FE0E1CF0C9DE3800CA50D12
:102B600071EDC128F9BA510D2B23EFED211608EBB9
:102B7000DD08BFF2FE094B00C2E47721EFEB430210
:102B8000A31631F015FEB60B6BF3FAF1251A71ECB2
:102B900085F0CC1F200847EAA608DA020EE51222CB
:102BA000A40022EA4B17F6F308ED510D410B7BF818
:102BB000BDFE27FABEF8EB00AD110801F1F489075C
:102BC00051E5EB16E80CFAF4CF0DDCE35A0CF0F902
:102BD0000C02640492EF062110EFB5FA61FFF1F4E4
:102BE0008C0F9F0189062EEBAA08630713F3361892
:102BF000EEEF1FF7490C7FE64811922F90CC0CECBA
:102C00004D36C2E49CFD3FFF6AE3F9254A067CE0AD
:102C1000BD01C320A2F498E3DE19C2F958FEF10BFE
:102C2000BAE2B8045A1FE0F9AAF2450B75EF8DF22B
:102C30007518D50310EF940E651140E4A400660DDD
:102C400046F11210980FF2DE2BFAF00EC5E9A71824
:102C5000D504F7D7490CDB121B0C51F7E00CAF047D
:102C6000D3E648100DE99702B71CF4E7CD00FD0E3E
:102C70002DEF0AE3031C230D40E55014BEF738F690
:102C8000A717AEF702F87C0B4B02EAF1CC05100255
:102C9000FCFDAE0933FC27FB1BF56AFC09FFE713BB
:102CA0009A0638E2BC03AD0F1FF7B000300E17F6DE
:102CB00096072FFBEEF0C21197FE51FA00FF960423
:102CC00039F588F7C917E203FDF8B9FC28F2CAFB09
:102CD00019180C0442EFE90900FFD6016B0CB2F49D
:102CE000E6F0B0026C0365FC950CB1FE8BFB35077A
:102CF0000DFF99F641F3FB02D6016F0D9509F7ED33
:102D0000910A9E0813F59301C0F0A8003E047008D4
:102D1000460833E8230C16FC65FF331493E89EF451
:102D2000C309DF110D00ED084FECB4EB7F270BF466
:102D300090F9ECFA7F0F6A0E42DB140519010F1DA2
:102D4000F7EFD1EE5F07E1F25319CEE7841FD8F712
:102D500029EFE40F3AD80A25C2FC16F9B709000298
:102D600070F3DA01A61D17E11114D5EF04ED3F143D
:102D7000DD072BFC0EFA33146BE22213F3FF5EF631
:102D800037FC09FBFF1A05E96515D5EEAB079CFE7C
:102D900001F97AFFF9E145378DDD5A1FA4FE9EDE69
:102DA000891DB6E47A117BE4112921ED95F493296C
:102DB0007FCD1127B9E911FDCA1075EBE10722E8B3
:102DC0003E2DB3F15400D40C34E1160FE8E4D323C4
:102DD00028F65703A50EA9E2FC1404EA2F11EDF51D
:102DE000BF0C9DF864F0761394E4881F1FF76FF70B
:102DF000F303CD01140356F43616FEF5A4001CF1BE
:102E0000B402081832EECB0F1BF5D4F5A1F8DD079C
:102E1000F50C75EFD02055E767F3CD00B5108A1596
:102E200040E78E161DD8BC026913BBF3D71104000E
:102E3000B60B2CE04B05C5004CFC0C17FFEE4E0BFF
:102E4000A3EE26FE3B019717BEF886D67F3B6DD8D2
:102E50000AF7B92652F2AC0114F2871303EFEBFE26
:102E60003C0D6EFC9B0043013B01A0E86017710024
:102E7000C2F9E00FCFE1C102A10EBBF52409A50CF8
:102E8000F8E8A1F9181AADE3DC0B2325E3FCDAD549
:102E9000DBE7B2372FD1900F663B3EC5750276FE59
:102EA00041F4D229F8FB76E95B1E33D0F3002226E9
:102EB00066E3B331FCD568EF5A1F7FE35E2453F11C
:102EC00012F8A8120DE630F47D2E55FCABDAE11EA7
:102ED00023E1DE17C40677E2772125DB0A0EF4131F
:102EE000E5F28908D9F2C8F38F15690028F2AB1A08
:102EF000ABD9840BFA1D68D8BF1E54019ADC780A3E
:102F0000340F40FC390B8F00CDEB310904ED1A0F63
:102F1000840DA6F4140767DF5C19780AA1F9A90EDD
:102F20005EE3CAFBD6157BF7A7EE631DC9EC600014
:102F3000211835F1AF08C1E83D0BF60735F1900FC8
:102F400038F66001E907B0EC990BF00EFAE0BF0B20
:102F50009300FBEE1A26D2FFB0EAB70807F048FE4E
:102F60008C22E6EE98F912FBF6F05028C5EA94FAA6
:102F700011152ED4791A6C1D57DB410BB70A7FE669
:102F8000ED0C700750FD150231F0F208A1F65A0D54
:102F9000D90381EE662272D2CFFA9B2A9BE99B006D
:102FA000BC06D3FB36EFF11F01FD38E45A1F03EFD7
:102FB000CEFD1B0B9CFB72FD49F70D1116FDF0FABF
:102FC000290747EB40111E1045E2E7119F01EFE989
:102FD000A10F76FF01F9D40BB2F940F9800C26FF5E
:102FE000710361FDFDFB33FC6FF682139CFE60EF05
:102FF000441339F5A9F9551111EC410A2C0C7DED5A
:10300000FF056A0FBCEC8CF7AC147BFBBF0841F7E3
:1030100062F6910828F49D0D24F46F0A280853DA0B
:103020000525A4FF68ED971708EDC3F64811530274
:10303000B3F0B01830F8B2E1E11DA0FB67F5D40B96
:1030400000012BF9F5F7450BCEFBB1FBC20E38F7AB
:10305000E602C101E9F2170B530430F5CEFCF50B83
:10306000E9F201FCD31102F7C90126FFDFFAAB0335
:103070009A04BC02F1F4B70A50FED1ED421A7AFC70
:10308000D0F12B10D8F6F9F981054B01BDFCF208FF
:1030900077F61BF586155DFB61FC3202B803EF0184
:1030A0000FF33313B6F638F6900E1DED4F174CFEA6
:1030B000EBE9620E51FA000187FE780A26FDFAF16B
:1030C000C70A2A0211002601DFFD30F9FF0454016E
:1030D000ECFA5911E9F3DAECFC1172FE61FD5B06C2
:1030E00002F8E3FF6002B5FD1B0B3105CFF6C90105
:1030F000C101B70718F07AEA120E83FD670A4D0E78
:10310000FBEF1A0F5000FCE9BF0BB6F9CCF29203AB
:103110004206560C0C04820045F50AF9730B02F7BF
:1031200067F33B14EE0419EC001783FD91F30D12C5
:103130003DDFA316240814D9D51BF70205FC47036D
:10314000A301A0FEAAF5ADFCB5FF9826DDF261D083
:10315000FB18C72080F58AEBC70A34FA01FCE700A8
:103160000DEB262BF20675D69F174F03E1F1FA07F8
:1031700084F5C9032B0F3CE34204AC2ACCDF09FCE5
:1031800096197CE1A50EFCFF26EA4922A9FBB5E6CB
:103190002A16F303B1E70A0C7007BBF1A608ECF896
:1031A000EDF6251909FEC9ED1C1BB2F907DE631DFA
:1031B000D90496F0401160EF8F006111D6ECE40D58
:1031C000AF070EE2A3044F050402D80DC4F08F0030
:1031D000C20F9BED83FAE218E8FB8FEBFE08580262
:1031E00009FD2AFEFEF4CF0F890897EB78065110EF
:1031F0004CEAB803C11602F5A20A01FA8BEA501490
:1032000099F625EE25189CFC57EE980E0305C10192
:103210002D076DEC16F9270F78F44B02291AFEF2F0
:1032200013F6410C5AF88BFD6803FDF8AF079E09B1
:10323000AEF3EA035F071DEED2FD14057E007D03A9
:103240009CFB2506FD0E66FA77F8310853EEAEF3C7
:10325000300E93FE5A0EB000B8EC4D106D020CEC1F
:10326000E2020C0580F6BF0B8C0CB9FB3604E9F2C8
:10327000E9F3FA0A09FF35F4A6090F09C2FB6F0A40
:10328000DFFDD4F4EBFD8DF4AE09F81089F1BC023A
:103290008D094EF5B7070001A6F63605A2F205FD29
:1032A000DD1C33FCB8EEFE082AFE2BFD180430F9B5
:1032B000F2052D050BF31003340E20F3E3FC940FFD
:1032C00023F733FB150209FFC407EF0033FB6C043F
:1032D000CAFD20F474068104CEFD21036AFAEFFFD3
:1032E0002D04D3F9EE053108F3EC6D015A0EE1F02F
:1032F00078098D0A9AEF3E0593FEB9FCCF0FC5FE03
:103300009EF447032E011FFA100544FC4704BC033A
:103310000BF2830EAB07CDEC3700F60997FEFF03E7
:10332000150134F5180443001BF70F0AB0015AF7D2
:10333000A70336044F02A303FDF70FF6CC067AFF6E
:10334000C1FF390787FCCEFFC4048A0159FC99F6F6
:10335000A0FE300B9CFC7FFAD80869FD83FA3A0482
:103360004B030D0016FC2CF76C03730D3CF8100397
:103370004D0DC6E711009C117FFCFDF932EBEC10FE
:103380000A206EE66EE62820A20A53DCDA00311A23
:10339000660D2BE468ED0E23C006CCDD2A01E52086
:1033A00078F559E7EE040620EA0524C996066D2D46
:1033B0002EEAF3EB2E17E90832EE2FFD2E039010C4
:1033C000DCF55BDD6224A10C4BEB880E4AF424F69D
:1033D000A81434F801E74A1E380FCAD46DFFA92398
:1033E0009B0152DF3CF92F2531052ED69E0850292E
:1033F000B1E823E1971541200DE9E3D3851C06369A
:10340000C5E967CA4C269B181BCC7903F025F10B44
:10341000BCD8A6DEE037B817C0C47006CE2875EB5E
:10342000DCE1FB04033137FDE1C5340F82298DF364
:103430008CE4840B141B1AE58CE09424BF1ED0DFAF
:10344000D3E61C1AB514B1E83EEFA21CF30280DDEE
:10345000B305301F560841E18DF401250AF81FE439
:103460005414A2095FF21BF56003CF2159FAB5D2BB
:1034700081186D1774DE7E01C5150DFD2AEAD3FB98
:103480006B1E9E057BE522FC4715AF043BE897FECB
:10349000B819A5F79FED2B0FF609DDF3B3F2D105AF
:1034A000E2195FF061EA3E1A14066BF36AF8E1086C
:1034B00098126EE868EDBB206405B5E5170A700840
:1034C00044FAECFA48FC441311FD4DE3A2084A1DEE
:1034D000E8FBA9E6B000E216E4F814F0840D8908D0
:1034E0002DF053EF0418471772E90CEFBA1092034E
:1034F00018F36402E604740947EAB1FBCC1ED7F85E
:1035000007F4BDFC57042504CFF93FFF8F110FF6D8
:10351000ACEC7115890788F63CF8EF000A0CD2FC78
:10352000D0F59010C6FBCDEE240A6707B4033DF238
:1035300049F966101100DFFAD505690177FA4FF0F5
:10354000E10897145FF3AFF07807B7095DFC8CF7DB
:103550004E06450B9BEA22FD1D1733FC03F12A02A0
:103560005F06D00745F78CF8A41249F7E1F4A303EE
:103570005E0C1D0270F0A703730C30F5ECF9410AE4
:10358000AF0477F824F4900D3203B7F043FF312FE6
:10359000C903E1C96CF0281FC22424DD9FEDD30FBD
:1035A000940D2D04EADA8D0A552574DE45F70B1FBC
:1035B00011EB6002F2070EF74D0DB4ECEF02141B95
:1035C000B0ED74F0E6016A11F30339F24B038200A7
:1035D00099F4F606A90F44FC8200A3ED0306F81245
:1035E000DDF35B0802F8D0F4D90583FCE617C2F9D5
:1035F000ECE4B01604012BFB280A95F4E3FE200648
:103600003AEF58145B0866E6C806B0FFFF034302B2
:1036100019FFE7001AFC7AFC840A5401F1F6DBFD7D
:1036200055F98C0F79012CF7A206E7FF3DF45304FE
:10363000300E0C02D4F2F6F39D0E470161FFEE0549
:10364000AAF5E605C3F7A800681925EED1EFBF0873
:1036500020086DFF9B003BFE22FFCAFD63F20513AD
:10366000390B19EE23FB53026B09110116F99A0766
:103670001BF9C7F72D050B06FB052CF55EF79D0D15
:10368000A302A6F3C8086306BBF554FD80084E07E5
:1036900030F9F1F5D009C1FDBEF98E0469FD7C0B4E
:1036A000C7F4CFF7F715BAF614F2520CD503E200BF
:1036B000C2FC0DFC670BA5FB6FF65E0B680351F8AF
:1036C00048FA1004340FC4F15EF9C809DBFB190194
:1036D00086FF8E05C900FEF39701941027FB80F446
:1036E000B3069B00ACFF8BFBB001020D7DF04DF9E2
:1036F000490D03067EFE10F1D9068E0567F46806B3
:10370000740945F5A5F881076707790334F551FB7E
:103710009D0D2FFA6AF9B20D72FC34F912FA5609AE
:10372000BF0918F298FB3E049A08B9FDC6FC2D05A6
:1037300054FFDDF281043313BAF928F2B400CC0946
:1037400087FE83FD10057101D0F383FD7B0FD90344
:1037500088F8DDEF1309DC0C3CF88105D2FCADFCE8
:103760002BFDB00295092BFCD3FB40F9D4090803CB
:1037700095F5DE027C08C2FB25EF1B0DFA0A4EF51B
:103780002101F5F9DD043D0830F7890526FF34F7FE
:1037900043038D0912FCE0F53605A7045CFFE8F948
:1037A0009B009A0594FBF3FFDAFFEE07B40121ECCE
:1037B0007F0E350863F579033BFDC005E3FB62FA34
:1037C0009A067C076FF891F60E0CEBFD55FBDD04B5
:1037D0007E0187FE94FAB404F700ADFDD6016DFEBC
:1037E0002105ECFAFDFAF20883FCECF90F08D80980
:1037F00073F713F33507D1031AFE740558001AFB4B
:1038000098FCCEFEC0069607E4F7ECF936028E046B
:10381000AC02B9FBCEFFA4FE51FAA206630683FBFD
:1038200015FE26FD1308CD03A2F54303CC065AF47A
:1038300038F8E40D060B6AF8A7EEA3033D0AE6028A
:1038400004022CF4DBFD9604D601FE09A5FA8DF1E5
:103850009B033109190161FE40F8D007340D77E36D
:1038600082FF4121CCF27EE9BB09880B65FD7EFF1A
:10387000D3F8C5FE4607A9FA8905950981F1ECF848
:10388000C807BC032809BEF89AF0E5091C0622FC0B
:103890005F09E9F66BF3BF0A1002F605E7FE08EFD1
:1038A000D4089109E9F6AF04D50680F309FDF205C5
:1038B0009F010E0E1BF5B4EEC20E9B038DF5C807DB
:1038C000790436EE8D06240890FBC9044EF5D1022A
:1038D000AE0D06F8F8FE81061FF797FE7405E201AB
:1038E0004B05BFF387FA5E0E00FE76FD0804F5F582
:1038F0002AFF810726FED009F0FB3FECD0085D13BC
:103900005EF6D3F8DC0966F953042FFC2502441057
:103910003FEC56F68908E50647FF76FC22FF66FB7A
:103920000306B8052006B1FA1EE899097F2494FC25
:1039300037E67BFB4B052006A8FE4701D10246EF88
:10394000A0FCB111A304BFF39CFBE1092FFCE7FE2F
:103950007501C1014A0AF4E99B004F1935F165FC74
:10396000BB088BFB27FC0400C80586036BF5B2F887
:103970002B0FA4FF3CFBA8015DFD5B072BFA76FF34
:103980005F0538F93605FF04A1F6CEFE8E018E02E2
:103990006C07D4F372FA3D0B9202E7FC66F7D5028E
:1039A000170CBEF933FE7101FCFDEE0550FCBDFFA6
:1039B000920448FB00FE2905CAFC43FFC10172FBCB
:1039C0003908F0FAF5F9510D83F9BEFA960533FF7F
:1039D0008D061EFC1AFA8907150137FCF8FF9A04B8
:1039E0002FFE77FA1100A703100398F9CAFC1F0BEA
:1039F00067089BECE9F629184F0374F248FBFF05B2
:103A00005F05F4FB1900D50472FD98FAB0FFFF02C0
:103A100047016EFB7807A4FFFAF326FFA414EB011D
:103A200052DFC6107D18B6E41CF4512401FDC8DD38
:103A300055105D102AFE2AEBE4F8DB26DDF0DED916
:103A40003C26D7118EDAFCFDC515C405EBFEA8E8AF
:103A5000F10C660FAADF9618140458EC9A0893FD2F
:103A6000000010054702A6F1800AB5FBF0F94717E0
:103A7000CFF717F51D0186FFCC07F608AFF2F5F872
:103A8000230DA5FB2103F30260EEA4136C034DE2AA
:103A90007A13D00A68F0D907D2FC23F7331334F530
:103AA00078F55C162DF12AFF9E05E8F89108B1FA29
:103AB0009BFF700547FF52F4730D7005EEEF5F0832
:103AC000CAFB10069CFDD7FB520AF4FA61FE33FED6
:103AD0003506D4F6E602770E9BED4F029E09DBFA1F
:103AE0008BFCC5FEB7064B025EF805FC8B1034FA62
:103AF000B8EBB915100353F06003DFFCFE0ACD00EC
:103B0000FEF41C05E106C1FD24F4E21761FF4EDD61
:103B1000D409FC132D0556F47CF50DFFAA0AFCFD13
:103B20004B014D0EB9E8B5FB280C6306D905EBEC4B
:103B3000DBFBBA107BF9CD01C212BCEEBCEE3E0736
:103B4000B20CAA0CE5F53EF0FB0509FF3E07C503E4
:103B5000630640F996DB1A25ED0AB7F0EA06B7F0DE
:103B60003109B6F8950A100505FC44FC7AE9D41D24
:103B7000E70078F51501CFFAA60B0BF2471599F877
:103B800008EB6D14F2F0E713D80A28E183FDD00AA0
:103B90003908D2FDEE0753F153ED7518AC012C092D
:103BA000A5F787E722114301F10B4AF42E034E09D2
:103BB00066E2A71743FE37FD8E011CF0F90FF1F8FE
:103BC000EA047902BDFEDE0364EFBE106C0545F623
:103BD0008BFD84F8270FF0FC7C09E4F6BDEAC01ADF
:103BE000EAF01B0E5F052BE5A50DBDFE5B08F0FAA4
:103BF0005704E0F849F77E1217F8730C18F295F69F
:103C00001A0FD6FDEA0373F9D40A02F4B6F8F90ED6
:103C100027FA4E0BD0F1DFFA0A0F87FADA0061FCBF
:103C2000E507E0F9A9FB830F98FBFDF9E8F84109E6
:103C3000E602DFFC520757EE4703A70569FE620F55
:103C4000A2F140F8B002A4002C09EFFEAF0496F1F7
:103C50008BFDED0C8A00180452F35401A4003F02BE
:103C6000A70412F93A0539F54E08460874F0E5083C
:103C7000A8FD50FF1B0A40F9150216FB72FC320426
:103C80003E03A70634F840F811FD200A2E01580023
:103C90006002F3ED1B0B530215FFC70AD9F0A4FF16
:103CA0004B045F05930145F8290412FCE6010C045E
:103CB00051FBDAFF6D0015FEA4FE7407C6FA48FC3E
:103CC0009A0591F65707B80559F9850462F93A0340
:103CD000CD028F00D104E1F0B708030462F99A081D
:103CE000E3FE52F4E7FC16121AFA080172FD42F1E3
:103CF000541383FC76FC5B08ECF9F9F904022F0FEE
:103D0000BBF5CFF85F0801FBE10758FEA1FA4B03B2
:103D100026FEC6FD8A02C30A5BF237FDF6082BFCBD
:103D2000310727FCCAFECEFBC5FF9A08A5FAB305EA
:103D30003200C8F24204BB0905FADE01D5027CF468
:103D4000A206B30673F65306B9FD17F8A50C93FF48
:103D5000A5F922FE36024B0482FEEF0188F91EFF10
:103D6000C40405FE35062600A5F73BFE3108C9014F
:103D70001AFA4F043FFD26FE5C0208028603A1F9F1
:103D8000370027FBA3044F056FF64A0993FD56F64B
:103D90002103670704FF2AFE65FFB6F5B307680431
:103DA000F6063F0068ED1D04AF0782FF5DFE61FE71
:103DB000B5FF5DFC9A04780902F6BAFA1C063BFFCF
:103DC000250398FC22FE9605CEFC4CFBC007E601BD
:103DD0006AF97AFFF301200651FA48FBE204470131
:103DE000B0FF8F0093FD51F8950A310861FDB9FECF
:103DF00010F087FC6114E204F30189F33BE74718F4
:103E00005B0644FD0E0F50EBABF18909380CA2089C
:103E1000B0021EE8A9FBAA0BADFDA013E4F8C3F3A2
:103E20002FFACAFC08195800F1F406F7FF7F627FE9
:103E30008A7D7D7A4276E3706E6AF262825A3451EC
:103E40001D47573CFC302825F9188C0C000074F3F2
:103E500007E7D8DA04CFA9C3E3B8CCAE7EA50E9DA0
:103E600092951D8FBE89838576829E8000809E807C
:103E700076828385BE891D8F92950E9D7EA5CCAEE0
:103E8000E3B8A9C304CFD8DA07E774F300008C0CB9
:103E9000F9182825FC30573C1D473451825AF262EC
:103EA0006E6AE37042767D7A8A7D627F00008C0CB8
:103EB000F9182825FC30573C1D473451825AF262CC
:103EC0006E6AE37042767D7A8A7D627FFF7F627FD1
:103ED0008A7D7D7A4276E3706E6AF262825A34514C
:103EE0001D47573CFC302825F9188C0C000074F352
:103EF00007E7D8DA04CFA9C3E3B8CCAE7EA50E9D00
:103F000092951D8FBE89838576829E8000809E80DB
:103F100076828385BE891D8F92950E9D7EA5CCAE3F
:103F2000E3B8A9C304CFD8DA07E774F3110000009F
:103F30001200000013000000140000001700000031
:103F40001800000000000000010000000000000058
:103F50000000000000000000000000000000000061
:103F60000000000000000000000000000000000051
:103F70000000000000000000000000000000000041
:103F80000000000000000000000000000000000031
:103F90000000000000000000000000000000000021
:103FA0000000000000000000000000000000000011
:103FB0000000000000000000000000000000000001
:103FC00000000000000000000000000000000000F1
:103FD00000000000000000000000000000000000E1
:103FE00000000000000000000000000000000000D1
:103FF00000000000000000000000000000000000C1
:0440000000000000BC
:04000005080000ED02
:00000001FF
